:100000000C942A000C9445000C9445000C94450077
:100010000C9445000C94B7010C94E4010C940F026D
:100020000C9445000C9455010C9445000C9445002B
:100030000C9445000C9445000C9431030C9445003D
:100040000C9445000C9445000C9445000C9445001C
:100050000C94450011241FBECFE5D4E0DEBFCDBF18
:1000600010E0A0E6B0E0E2E3FEE002C005900D92F1
:10007000A43AB107D9F710E0A4EAB0E001C01D929C
:10008000AF3FB107E1F70C94B1000C940000CF939F
:10009000DF93CDB7DEB7E7E3F0E08FE18083E4E301
:1000A000F0E08EEF8083E1E3F0E084E08083E2E340
:1000B000F0E088E38083DF91CF910895CF93DF93C1
:1000C000CDB7DEB723970FB6F894DEBF0FBECDBF16
:1000D0008091AF008823E1F31092AF0080E29EE4AC
:1000E0009093FC008093FB001B822FC08B81482FD4
:1000F00055278B819927880F991FFC01EE53FF4FDD
:10010000808191819C0128513C4FCA01880F991F21
:10011000FC01E551FF4F318320832091FB0030919A
:10012000FC008B819927880F991FFC01E551FF4F37
:1001300080819181A901481B590BCA019093FC0051
:100140008093FB008B818F5F8B838B81883070F273
:1001500023960FB6F894DEBF0FBECDBFDF91CF91CF
:100160000895CF93DF93CDB7DEB727970FB6F894F6
:10017000DEBF0FBECDBF0E9447000E9433010E9428
:1001800023030E9472031092E9008EEC92E0909398
:10019000BD008093BC008CE193E09093BF008093FE
:1001A000BE0078948091A8008823E1F31092A80003
:1001B0000E941B060E945A040E94620600C08091A1
:1001C000AB00813011F40E948B068091A900813030
:1001D00041F41092AA008091E900882311F40E9452
:1001E0005E008091A800813019F51092A8001A8253
:1001F0001CC080E690E00E94AC038A8199270E948F
:10020000F60387E690E00E94AC038A819927880F65
:10021000991FFC01E551FF4F808191810E94F603F7
:100220000E94E7038A818F5F8A838A81893008F37D
:100230008091A700813019F61092A700C0CFCF930C
:10024000DF93CDB7DEB7F894E9E5F0E089E180838C
:100250007894DF91CF910895CF93DF93CDB7DEB738
:10026000DF91CF910895CF93DF93CDB7DEB7E3E56C
:10027000F0E082E08083EFE4F0E01082EEE4F0E072
:1002800082E08083EAE4F0E084EF91E09183808370
:10029000E8E4F0E080ED97E091838083E9E5F0E029
:1002A00089E18083DF91CF9108951F920F920FB65D
:1002B0000F9211248F93CF93DF93CDB7DEB7809148
:1002C000B3008F5F8093B3008091B300883029F42E
:1002D00081E08093AB001092B3008091E8008F5FC3
:1002E0008093E8008091E8008834C9F581E080932C
:1002F000A9001092E8008091B2008F5F8093B20055
:100300008091B200853029F41092B20081E0809390
:10031000AA008091B0008F5F8093B0008091B00000
:10032000843641F41092B00081E08093A60081E011
:100330008093A8008091B000823319F481E080930B
:10034000A8008091B1008F5F8093B1008091B100CF
:100350008A3029F41092B10081E08093A700DF91E8
:10036000CF918F910F900FBE0F901F9018951F92F5
:100370000F920FB60F9211242F933F934F935F93D9
:100380006F937F938F939F93AF93BF93EF93FF935D
:10039000CF93DF93CDB7DEB7E091BC00F091BD0005
:1003A0000995DF91CF91FF91EF91BF91AF919F910F
:1003B0008F917F916F915F914F913F912F910F900E
:1003C0000FBE0F901F9018951F920F920FB60F92AD
:1003D00011248F93AF93BF93EF93FF93CF93DF934A
:1003E000CDB7DEB7A2E3B0E0E2E3F0E080818B7F3F
:1003F0008C93A5E3B0E0E5E3F0E080818D7F8C9302
:1004000081E08093AF00DF91CF91FF91EF91BF9199
:10041000AF918F910F900FBE0F901F9018951F9264
:100420000F920FB60F9211242F933F938F939F93A8
:10043000AF93BF93EF93FF93CF93DF93CDB7DEB727
:100440002297DEBFCDBFA2E3B0E0E2E3F0E080811F
:1004500084608C93ECE4F0E011821082A8E4B0E0B8
:100460008091A4009927880F991FFC01E551FF4F47
:100470008081918111969C938E938091A400882312
:1004800039F4A5E3B0E0E5E3F0E0808182608C938D
:100490008091A400282F33273A83298389819A8168
:1004A00082309105C1F129813A812330310554F41C
:1004B00089819A81009789F029813A81213031051B
:1004C000D9F04EC089819A818330910599F12981B3
:1004D0003A8124303105E9F143C0A8E3B0E0E8E314
:1004E000F0E0808180618C93A8E3B0E0E8E3F0E085
:1004F000808181608C9334C0A8E3B0E0E8E3F0E051
:1005000080818E7F8C93A8E3B0E0E8E3F0E0808107
:1005100082608C9325C0A8E3B0E0E8E3F0E080813E
:100520008D7F8C93A8E3B0E0E8E3F0E08081846005
:100530008C9316C0A8E3B0E0E8E3F0E080818B7F05
:100540008C93A8E3B0E0E8E3F0E0808188608C93CE
:1005500007C0A8E3B0E0E8E3F0E08081877F8C93F8
:100560008091A4008F5F8093A4008091A4008930C3
:1005700010F01092A4002296F894DEBFCDBFDF9158
:10058000CF91FF91EF91BF91AF919F918F913F914B
:100590002F910F900FBE0F901F901895CF93DF9360
:1005A000CDB7DEB78091B4009091B5000097B1F45B
:1005B000E6E4F0E0808191819093BB008093BA00E3
:1005C000AEE4B0E0EEE4F0E080818F7B8C9381E0DC
:1005D00090E09093B5008093B4002BC0E6E4F0E087
:1005E000808191819093B9008093B800AEE4B0E02F
:1005F000EEE4F0E0808180648C932091B80030912B
:10060000B9008091BA009091BB00A901481B590B19
:10061000CA019093B7008093B6001092B500109273
:10062000B4008091B6009091B7009093FE00809343
:10063000FD00DF91CF910895CF93DF93CDB7DEB763
:10064000DF91CF910895CF93DF93CDB7DEB7E7E287
:10065000F0E01082E6E2F0E08FEE8083DF91CF9150
:1006600008951F920F920FB60F9211242F933F936C
:100670008F939F93EF93FF93CF93DF93CDB7DEB725
:10068000E6E2F0E010828091A5009927E4E2F0E034
:1006900020813181880F991FFC01EE53FF4F318378
:1006A00020838091A5008F5F8093A5008091A50095
:1006B000883010F01092A500E7E2F0E08091A500EC
:1006C0008083E6E2F0E08FEE8083DF91CF91FF91AF
:1006D000EF919F918F913F912F910F900FBE0F90AF
:1006E0001F901895CF93DF93CDB7DEB7E9E2F0E026
:1006F00080E18083E0E4F0E01082EAE2F0E088E16B
:100700008083E0E4F0E086E88083EBE2F0E082ECD6
:100710008083DF91CF910895CF93DF93CDB7DEB77C
:1007200021970FB6F894DEBF0FBECDBF8983EBE2F1
:10073000F0E080819927807290700097C1F3ECE21D
:10074000F0E08981808321960FB6F894DEBF0FBE5A
:10075000CDBFDF91CF910895CF93DF93CDB7DEB7B3
:1007600026970FB6F894DEBF0FBECDBF9E838D8354
:100770008D819E81DC01FD0101900020E9F7319718
:10078000CF018A1B9B0B9C838B831A8219820FC01B
:1007900029813A818D819E81F901E80FF91F8081BD
:1007A0000E948C0389819A8101969A838983298189
:1007B0003A818B819C818217930750F726960FB65A
:1007C000F894DEBF0FBECDBFDF91CF910895CF93D8
:1007D000DF93CDB7DEB780916A000E948C038091D1
:1007E0006B000E948C03DF91CF910895CF93DF932C
:1007F000CDB7DEB766970FB6F894DEBF0FBECDBF9C
:100800009E8B8D8B8D899E894AE050E09E012F5FE3
:100810003F4FB9010E94D406CE0101960E94AC035D
:1008200066960FB6F894DEBF0FBECDBFDF91CF91B5
:100830000895CF93DF93CDB7DEB722970FB6F89424
:10084000DEBF0FBECDBF8A8387E089831FC08A8148
:10085000482F55278981282F332727FD309581E0A0
:1008600090E0022E02C0880F991F0A94E2F78423B9
:1008700095231816190624F481E30E948C0303C003
:1008800080E30E948C038981815089838981882338
:10089000F4F680916A000E948C0380916B000E94A4
:1008A0008C0322960FB6F894DEBF0FBECDBFDF914A
:1008B000CF910895CF93DF93CDB7DEB70E94930415
:1008C00063E080E00E94F7058CE690E00E949905C5
:1008D00062E081E00E94F70587E790E00E949905B9
:1008E0000E948904E0E3F0E0808199278072907093
:1008F0000097C1F70E949304DF91CF910895CF93A1
:10090000DF93CDB7DEB78DE00E94CE05DF91CF91AA
:100910000895CF93DF93CDB7DEB78CE00E94CE056C
:10092000DF91CF910895CF93DF93CDB7DEB781E00C
:100930000E94CE05DF91CF910895CF93DF93CDB77D
:10094000DEB726970FB6F894DEBF0FBECDBF9E83ED
:100950008D838AE090E09C838B831CC082E390E0CF
:100960009A8389830EC08D819E8101979E838D839A
:100970008D819E810097B9F789819A8101979A8329
:10098000898389819A81009799F78B819C8101974E
:100990009C838B838B819C81009701F726960FB6F1
:1009A000F894DEBF0FBECDBFDF91CF910895CF93F6
:1009B000DF93CDB7DEB721970FB6F894DEBF0FBE39
:1009C000CDBF89838981992781709070882341F0F8
:1009D000A5E3B0E0E5E3F0E0808180618C9307C09F
:1009E000A5E3B0E0E5E3F0E080818F7E8C93898120
:1009F000992782709070009741F0A5E3B0E0E5E39D
:100A0000F0E0808180628C9307C0A5E3B0E0E5E36D
:100A1000F0E080818F7D8C9389819927847090701C
:100A2000009741F0A5E3B0E0E5E3F0E08081806469
:100A30008C9307C0A5E3B0E0E5E3F0E080818F7B15
:100A40008C938981992788709070009741F0A5E375
:100A5000B0E0E5E3F0E0808180688C9308C0A5E316
:100A6000B0E0E5E3F0E090818FE789238C93219655
:100A70000FB6F894DEBF0FBECDBFDF91CF910895C2
:100A8000CF93DF93CDB7DEB7A5E3B0E0E5E3F0E0C9
:100A9000808184608C9381E090E00E949D04A5E3B6
:100AA000B0E0E5E3F0E080818B7F8C93DF91CF9124
:100AB0000895CF93DF93CDB7DEB722970FB6F894A2
:100AC000DEBF0FBECDBF8A838A8182958F708983F6
:100AD00089810E94D7040E9440058A810E94D70420
:100AE0000E94400522960FB6F894DEBF0FBECDBF20
:100AF000DF91CF910895CF93DF93CDB7DEB72197E4
:100B00000FB6F894DEBF0FBECDBF8983A5E3B0E07A
:100B1000E5E3F0E0808188608C9389810E9459052B
:100B200021960FB6F894DEBF0FBECDBFDF91CF91F7
:100B30000895CF93DF93CDB7DEB724970FB6F8941F
:100B4000DEBF0FBECDBF9C838B838B819C81DC017C
:100B5000FD0101900020E9F73197CF018A1B9B0B23
:100B60008A8319820EC0898199279C018B819C817F
:100B7000F901E80FF91F80810E947B0589818F5F51
:100B8000898399818A81981770F324960FB6F89417
:100B9000DEBF0FBECDBFDF91CF910895CF93DF931E
:100BA000CDB7DEB721970FB6F894DEBF0FBECDBF2D
:100BB000898381E090E00E949D04A5E3B0E0E5E335
:100BC000F0E08081877F8C9389810E945905A5E39D
:100BD000B0E0E5E3F0E0808188608C9321960FB669
:100BE000F894DEBF0FBECDBFDF91CF910895CF93B4
:100BF000DF93CDB7DEB723970FB6F894DEBF0FBEF5
:100C0000CDBF8A836B838A81882319F48B818058B6
:100C100089838A81813019F48B8180548983898109
:100C20000E94CE0523960FB6F894DEBF0FBECDBF4F
:100C3000DF91CF910895CF93DF93CDB7DEB781E0F9
:100C400090E00E949D04A5E3B0E0E5E3F0E0808140
:100C5000877F8C9383E00E94D7040E94400585E043
:100C600090E00E949D0483E00E94D7040E9440050A
:100C700081E090E00E949D0483E00E94D7040E94DE
:100C8000400582E00E94D7040E94400581E090E088
:100C90000E949D0488E20E94CE058EE00E94CE054F
:100CA00081E00E94CE0584E890E00E9499056AE008
:100CB00081E00E94F70589E890E00E949905DF91A4
:100CC000CF910895CF93DF93CDB7DEB71092AE00EA
:100CD0000E94930460E080E00E94F7058EE890E0B7
:100CE0000E94990569E080E00E94F70586E990E09E
:100CF0000E94990560E081E00E94F7058DE990E08F
:100D00000E94990560E080E00E94F7050E947F0440
:100D1000DF91CF910895CF93DF93CDB7DEB72197C1
:100D20000FB6F894DEBF0FBECDBF1982E0E3F0E04E
:100D30008081992780719070009711F081E08983FC
:100D4000E0E3F0E08081992788709070009721F0AF
:100D5000898193E089278983998180916900292F6E
:100D6000281B822F89838981992787FD909581701F
:100D70009070882381F080916900982F8981890F74
:100D8000809369008981982F92708091EA00890F81
:100D900081508093EA0021960FB6F894DEBF0FBE13
:100DA000CDBFDF91CF910895FB019F01E8944230C0
:100DB000C4F04532B4F44A3029F497FB1EF4909500
:100DC00081959F4F642F77270E940507805D8A33A6
:100DD0000CF0895D8193CB010097A1F716F45DE2D9
:100DE00051931082C9010C94F506DC01FC010190BD
:100DF0000020E9F73297AE17BF0730F47C9160818D
:100E0000708331976D93F7CF0895AA1BBB1B51E1F7
:100E100007C0AA1FBB1FA617B70710F0A61BB70B6A
:100E2000881F991F5A95A9F780959095BC01CD010F
:020E3000089523
:100E32004B2000000000003D00010D0A4550492DE5
:100E42005465737465720056657273696F6E2030F3
:100E52002E3264006875687500416B6B75005050E6
:100E62004D2D4F75740050504D2D496E00444D5814
:040E72002D496E0098
:00000001FF
